:0400000508000000EF
:020000040800F2
:1000000000500020850B0008ED000008EF000008FC
:10001000F1000008F3000008F500000800000000EF
:10002000000000000000000000000000F7000008D1
:10003000F7000008F7000008DF010008C52D0008E0
:1000400071140008251300089113000845130008D7
:10005000C91200083513000855120008651200087F
:100060008912000899120008A9120008E511000879
:10007000F5110008051200081512000825120008E5
:100080003512000845120008B51100085114000887
:1000900061140008C5110008D5110008B912000844
:1000A000A1130008D1130008C1130008B113000800
:1000B000E1130008F113000801140008ED12000814
:1000C000D912000811130008FD1200086913000876
:1000D0007D130008111400082514000839140008C5
:1000E00075120008551300084D140008FEE7FEE7DE
:1000F000FEE7FEE7FEE7FEE700F002F800F0A1FBF6
:100100000AA090E8000C82448344AAF10107DA4572
:1001100001D100F096FBAFF2090EBAE80F0013F020
:10012000010F18BFFB1A43F001031847F842000003
:1001300018430000103A24BF78C878C1FAD8520793
:1001400024BF30C830C144BF04680C607047000051
:100150000023002400250026103A28BF78C1FBD8D0
:10016000520728BF30C148BF0B60704700F002BD86
:1001700072B6704762B67047EFF3108072B6704780
:1001800080F310887047B0FA80F0704790FAA0F0C2
:10019000704730BF704720BF70470000EFF31080FA
:1001A00072B6704780F3108870471D484FF6FF7194
:1001B0000170002080F309881A48012101701A4853
:1001C0004FF08051016062B6FEE717484FF0805152
:1001D0000160704714484FF080510160704772B65B
:1001E000EFF3098028B1203880E8F00F0F49096843
:1001F000086000B50E4880475DF804EB0D480E49D5
:100200000A78027009480D490A680260106890E88F
:10021000F00F203080F309884EF0040E62B670476C
:1002200020ED00E07300002004ED00E090000020CD
:100230001D2100087000002071000020980000209F
:100240002DE9FF5F4FF0000904460D464FF0010A0B
:100250004FF0800BC0F83C90E06A0768B84604E0B5
:10026000E06AE16B0768491CE163A16A8847060000
:1002700001D0252EF4D1B84504D03A464146204657
:10028000236A9847002E70D0A64F00267F44D4E9F9
:100290000A108847202807DB312805D2391811F8C1
:1002A000201C09B10E43F2E7C4F838900027C4F8C7
:1002B00034902A280ED101CD04EB87014863D4E99C
:1002C0000A108847012F26D1A16B00292DDA26F0CC
:1002D00020062AE0A0F130010A291AD2BAF1000F53
:1002E00017D004EB8708C8F8341008E0D8F83410A9
:1002F00001EB810100EB41003038C8F83400D4E94B
:100300000A108847A0F130010A2902D2BAF1000F81
:10031000ECD1012F09D02E2807D1D4E90A10884743
:100320007F1C022F46F02006C3DB616B002903DA35
:10033000494246F001066163F10701D026F010063C
:10034000B10701D526F004066C2801D0682813D126
:100350000746D4E90A108847B84207D158466C2F9F
:1003600001D04FF48060064316E08CE040216C2FF2
:1003700000D089000E4312E04C2805D06A2803D033
:10038000742801D07A280AD149464C2803D059460E
:100390006A2800D000210E43D4E90A108847652856
:1003A000A6616FD014DC4728FBD008DC00286AD097
:1003B000412869D04528F4D04628F2D01CE05828BE
:1003C00057D06128F5D063281DD0642874D013E07D
:1003D0006F2861D008DC6628E3D067287FD06928C1
:1003E0006AD06E2839D007E0702842D073281BD01D
:1003F000752861D078283CD0E269616A9047E06B4B
:10040000401CE06328E70122700606D5ADF806908F
:1004100001CD01A9ADF804000BE08DF8019069460B
:1004200001CD8DF800000EE002CD4FF0FF327006D6
:1004300009D5206B0028204602D0AFF300800BE7DF
:10044000AFF3008008E7206B0028204602D0AFF30E
:10045000008001E7AFF30080FEE6700504D4F005EC
:1004600002D4300600D47006204602CDAFF30080DF
:10047000F2E6310609D5ED1D25F00705D5E9002383
:10048000083504E02BE046E037E004CD4B4601465A
:10049000204600F06FF8DFE6300606D5ED1D25F0AA
:1004A0000705D5E90023083501E004CD4B46204679
:1004B000AFF30080D0E6FFE731060AD501462046BB
:1004C000ED1D25F00705D5E900230835AFF30080C1
:1004D000C2E604CD0146204600F0B4F8BCE6ED1DAE
:1004E00025F00705D5E900120835CDE902120146CD
:1004F000204602AAAFF30080AEE6ED1D25F0070509
:10050000D5E900120835CDE902120146204602AABB
:10051000AFF30080A0E6E06B04B0BDE8F09F704749
:10052000704770476041000070B50446456B8069B4
:100530003026C10600D42026C00709D106E0E269B2
:100540003046616A9047E06B401CE0636D1EF6D553
:1005500070BD70B50446456B8069C00709D006E0E0
:10056000E269616A20209047E06B401CE0636D1EE9
:10057000F6D570BD2DE9F04F07460D46104689B0FF
:10058000DFF8AC80F844582901D0A8F11108B96906
:10059000090602D504461E4604E03946AFF3008042
:1005A000002604460FF28C09B8694FF0000A0107D3
:1005B00016D5702D04D10FF280094FF0010A11E019
:1005C000002386EA030184EA030008430FD00FF2F8
:1005D0006C09782D01D00FF268094FF0020A06E08D
:1005E000702D04D140F02000B8610820B8630025C8
:1005F0000DF1040B0AE004F00F00240918F80000C4
:1006000044EA06740BF805006D1C3609002386EADF
:10061000030184EA03000843EDD14B462A463846DD
:1006200001A9CDF800A000F02BF909B0BDE8F08FCA
:100630008A3E00000000000040000000307800000A
:10064000305800002DE9F041074610460026752974
:1006500039468AB015A510D0AFF30080002802DA21
:10066000404213A507E0B9698A0701D511A502E048
:10067000490704D510A5012601E0AFF3008000244E
:100680000DF1080805E000F0B0F9303108F8041069
:10069000641C0028F7D12B462246384602A9009652
:1006A00000F0EEF80AB0BDE8F081000000000000A4
:1006B0002D0000002B000000200000000FB40A4AAB
:1006C0000A4910B503AB7944029800F02BF90446AF
:1006D000054800F046F920B14FF0FF3010BC5DF83E
:1006E00014FB2046FAE70000D41800204F39000020
:1006F0000FB409491CB506AB6A46794400900598C9
:1007000000F010F904460020694600F025F9204663
:100710001CBC5DF814FB00005B0200004FF00002FF
:1007200000B5134694469646203922BFA0E80C50E7
:10073000A0E80C50B1F12001BFF4F7AF090728BFC2
:10074000A0E80C5048BF0CC05DF804EB890028BF3E
:1007500040F8042B08BF704748BF20F8022B11F067
:10076000804F18BF00F8012B7047032A40F23180F8
:1007700010F0030C00F0158011F8013BBCF1020FE2
:10078000624498BF11F801CB00F8013B38BF11F863
:10079000013BA2F1040298BF00F801CB38BF00F87A
:1007A000013B11F0030300F0EB80083AC0F0098030
:1007B00051F8043B51F804CB40F8043B40F804CB1B
:1007C000F3E7121D5CBF51F8043B40F8043BAFF364
:1007D0000080D20724BF11F8013B11F801CB48BFBC
:1007E00011F8012B24BF00F8013B00F801CB48BFF2
:1007F00000F8012B704740EA0103024630B59B0721
:1008000010D14FF0013400E008C208C91D1B9D4300
:1008100015EAC41FF8D013F0FF0102F8011B0ED037
:100820001B0AF8E711F8014B02F8014B002C1346A4
:1008300005D011F8014B5A1C002C1C70F2D130BDB0
:100840007047AFF3008000F0FCF803B400F06BF9E0
:1008500003BC00F008F90FB400F06AF90FBC03F014
:10086000EDFB00F0E7F801B5AFF3008000F052F9BE
:10087000BDE8014000F002F86FF0000000F0BEF8A3
:100880002DE9F0478946044615469A468169DDF808
:100890002080880604D5A06B21F01001A16100E042
:1008A00001200027A84200DD471B606B79194144F5
:1008B000401A6063A069C00602D42046FFF734FEE8
:1008C000002608E0E2691AF80600616A9047E06BCA
:1008D000401C761CE0634645F4DBA069C0060AD5DF
:1008E0002046FFF721FE06E0E269616A302090476A
:1008F000E06B401CE063381EA7F10107F4DC07E061
:10090000E26919F80500616A9047E06B401CE063FA
:10091000281EA5F10105F3DC2046FFF71AFEBDE80D
:10092000F08700000FB50846194691B007900848B7
:1009300009927844089000200C90064878440A9068
:1009400011A80B906846FFF77BFC15B000BD0000B6
:10095000DB000000EB0000000A6802F8010B0A60EF
:10096000704770B5044600F13C052846AFF300809F
:10097000E06800F080042846AFF30080204670BD98
:1009800010B5203AC0F00E8021BFB1E81850A0E8A1
:100990001850B1E81850A0E8185028BFB2F1200252
:1009A000BFF4F2AF5FEA027C24BFB1E81850A0E8C0
:1009B000185044BF18C918C0BDE810405FEA827CD7
:1009C00024BF51F8043B40F8043B08BF7047D207EE
:1009D00028BF31F8023B48BF11F8012B28BF20F88F
:1009E000023B48BF00F8012B70474FF00A01B0FBF3
:1009F000F1F202FB110110467047000003494FF06D
:100A00001800ABBE70470000310100002600020054
:100A100070B505460C46164604E0EB6914F8010B68
:100A2000696A9847B442F8D370BD01684A1C0260F5
:100A3000087870470446AFF300802046FFF713FFA5
:100A40007047744600F07AF8A6460DB500F086F8B7
:100A50000400BDE80D4011007047020010B50020F1
:100A6000AFF3008010BD2DE9FE4304460D4603F0B0
:100A700011FB0020CDE90045102000BF0290684620
:100A8000FFF774FB04460D46DDE9000117461E46DC
:100A9000AFF30080AFF30080AFF300800021084681
:100AA000AFF30080804600F05FF800218146C0F877
:100AB00000800846AFF30080411CC9F804100021F3
:100AC0000846AFF300800021C9F808000846AFF3DC
:100AD00000800021C9F80C000846AFF30080C9F877
:100AE0001000AFF30080AFF30080AFF30080AFF3EE
:100AF0000080AFF30080AFF30080AFF30080AFF36E
:100B00000080AFF3008003B0204629463A463346C2
:100B1000BDE8F08310B50020AFF30080AFF3008094
:100B2000AFF3008010BD6FF000006FF0020170475E
:100B300010B5AFF3008010BD7047000004490348B2
:100B4000044A054B21F007018D4670470040002004
:100B50000050002000480020004800200148704755
:100B6000704700005C190020014870477047000082
:100B70006C19002070470000014870477047000062
:100B80008019002000480047F9000008002981680A
:100B90000CBF21F0010141F0010181607047002983
:100BA00081680CBF21F4807141F4807181607047CD
:100BB00001468968002011F0040F18BF012070471A
:100BC00001468968002011F0080F18BF0120704706
:100BD00010B4426891F804C022F4807222F47022AA
:100BE0000B6842EA0C221A43426082680B4B4C7934
:100BF0001A40D1F808C0CB6842EA440243EA0C0329
:100C00001A438260C26A097C22F47002491EC9B28A
:100C100042EA0151C16210BC70470000FDF7F1FFCC
:100C200070B5FFF7A9FA3E490A78521C0A70FFF71F
:100C3000A7FA022000F0B6FD00286CD0394C3A49E2
:100C40002078A1F16002401CC0B220700B88D2F85D
:100C500000C0A1F1A005A3EB0C03D5F800C00A2841
:100C600063442B60B1F802C05668D5F804E0ACEBE1
:100C7000060CF444C5F804C08E88D2F808E0D5F814
:100C800008C0AEEB060EF444C5F808C0CE88D2F812
:100C90000CE0D5F80CC0AEEB060EF444C5F80CC061
:100CA000B1F808C01669D5F810E0ACEB060CF444B6
:100CB000C5F810C05269B1F80AC06969A2EB0C020C
:100CC0001144696120D3281F05F11C0103224FF054
:100CD0000A0E00BF50F808CF93FBFEF39CFBFEFC0E
:100CE0004B60436841F808CF521EF3D100202860C2
:100CF0006860A860E86068612861A861E8612070A8
:100D0000606801F04FF803E00121084800F05DF849
:100D1000022000F0BBFCBDE8704000F0CDBE00003A
:100D20006E0000205C000020BC0B0020002401406D
:100D300030B4072509290CD9C468A1F10A0C0CEBC1
:100D40004C0C05FA0CF5AC4303FA0CF32343C360D7
:100D500009E0046901EB410C05FA0CF5AC4303FA18
:100D60000CF3234303614FF01F0C072A0CD2436B93
:100D7000521E02EB82020CFA02FC23EA0C039140A1
:100D80001943416330BC70470D2A0CD2036BD21F4C
:100D900002EB82020CFA02FC23EA0C039140194395
:100DA000016330BC7047C36A0D3A02EB82020CFA51
:100DB00002FC23EA0C0391401943C16230BC704726
:100DC000816841F0080181607047002981680CBF8B
:100DD00021F4A00141F4A00181607047816841F0D5
:100DE0000401816070470000024A1070114690684B
:100DF00000F02CBF00000020704701F033BE7047A8
:100E000030B5ADF5077D002400F080F801F0ECFF6F
:100E100001F012F84FF4E13001F004FD274801F031
:100E20005FFE01F0E7FD002000F07EFE24498860AF
:100E3000002000F031FF23490323086022480022EC
:100E4000802101AD0FC50B2300F5FE7200211F4864
:100E5000009301F00DF8069006AA1DA10B2001F0E9
:100E60006DF802F04DFC054601461DA0FFF726FC7B
:100E700055B907AA4FF40071002002F01DFD40B1E2
:100E8000014617A0FFF71AFC022000F00BFB192502
:100E900003E0012001F044F9EBE7641CB4FBF5F03A
:100EA00005FB1040002804BF022000F00FFB0A23BE
:100EB00000221146104601F065F9EEE7E90D000841
:100EC0000000002060000020EC080020DD3D00084C
:100ED0005465726D696E616C205461736B00000023
:100EE00073647265743D3078253032580D0A000005
:100EF000704701F0D1BD01F0F9BD00B585B068467D
:100F000002F0E0F9009805B000BD00002DE9F043C3
:100F100087B002F0B9F94FF4803002F053FA02F0D2
:100F20009BFA012828D1002002F042FA002002F0AA
:100F30006FFA4FF4806002F061FA4FF4004002F063
:100F400075F9022000F076FC102000F067FC4FF4E9
:100F5000E0114FF4803002F06BFA012002F062FAE7
:100F6000392002F005FA0028FAD0022002F06AFACD
:100F700002F016FA0828FBD1222000F0D9FA24202A
:100F800000F0D6FA292000F0D3FA002000F0D0FAC1
:100F90000121084602F054F90121480202F068F9E3
:100FA0000024774E8DF81B400F25ADF8185006A988
:100FB000304600F04BFC734FADF8185006A9384688
:100FC00000F044FC4FEA7639484600F073FB6F4866
:100FD0006D4901604FF008088460C0F80C8000F192
:100FE0004001046141608021416149008D00C5617B
:100FF0008161202101624FF44051846241620146C7
:10100000484600F0E7FB62490B2000F039FA0B205C
:1010100000F0C8F801220221484600F0D3FB01216C
:10102000484600F03DFB5B480121046001714471BA
:101030004FF46021C460816080F81080DFF858812F
:1010400001464046FFF7C4FD0023012219464046F1
:10105000FFF76EFE0222002311464046FFF768FEAE
:101060000322002311464046FFF762FE00230422BC
:101070000B214046FFF75CFE002305220C21404671
:10108000FFF756FE002306220D214046FFF750FED3
:101090000023072201214046FFF74AFE00230822D1
:1010A0000A214046FFF744FE01214046FFF777FD45
:1010B00001214046FFF76AFD4046FFF781FE4046AA
:1010C000FFF77EFD0028FAD14046FFF787FE404635
:1010D000FFF76EFD0028FAD10121102002F0C8F8B8
:1010E000C020ADF818004FF003088DF81A801020CA
:1010F0008DF81B0006A9384600F0A8FB4FF4E1303C
:101100000290ADF81040ADF814400C204FF4007779
:10111000ADF80C40ADF81200ADF80040ADF8047029
:10112000ADF80E40ADF80240ADF806402E2000F0BC
:10113000FFF9222000F0FCF9ADF818708DF81A8044
:1011400018208DF81B0006A9304600F07FFBADF893
:10115000185004208DF81B0006A9304600F076FBDD
:101160000E4C02A9204602F00CFF6946204602F010
:10117000ACFE0121204602F0BAFE07B0BDE8F083C4
:1011800000080140001001404C2401407C0B00206D
:10119000210C0008A80B0020002401400038014069
:1011A000FEF7E6BF2A283EBF1030C0B200F00CBAEE
:1011B000704700000248806C002818BF0047704745
:1011C000CC0B00200248406D002818BF0047704734
:1011D000CC0B00200248806D002818BF00477047E4
:1011E000CC0B00200248C06A002818BF0047704797
:1011F000CC0B00200248006B002818BF0047704746
:10120000CC0B00200248406B002818BF00477047F5
:10121000CC0B00200248806B002818BF00477047A5
:10122000CC0B00200248C06B002818BF0047704755
:10123000CC0B00200248006C002818BF0047704704
:10124000CC0B00200248406C002818BF00477047B4
:10125000CC0B002002488069002818BF0047704767
:10126000CC0B00200248C069002818BF0047704717
:10127000CC0B00200348D0F8A000002818BF00477E
:1012800070470000CC0B00200248006A002818BFFD
:1012900000477047CC0B00200248406A002818BF66
:1012A00000477047CC0B00200248806A002818BF16
:1012B00000477047CC0B00200248C06D002818BFC3
:1012C00000477047CC0B002002480069002818BF77
:1012D00000477047CC0B00200348D0F8800000285E
:1012E00018BF004770470000CC0B00200248C06FB9
:1012F000002818BF00477047CC0B00200348D0F8E7
:101300008800002818BF004770470000CC0B002061
:101310000348D0F88400002818BF00477047000039
:10132000CC0B002002484068002818BF00477047D7
:10133000CC0B002002484069002818BF00477047C6
:10134000CC0B00200248C068002818BF0047704737
:10135000CC0B00200348D0F8A400002818BF004799
:1013600070470000CC0B00200348D0F88C00002808
:1013700018BF004770470000CC0B00200348D0F88E
:101380009000002818BF004770470000CC0B0020D9
:1013900002488068002818BF00477047CC0B002027
:1013A0000248006E002818BF00477047CC0B002091
:1013B0000248C06E002818BF00477047CC0B0020C1
:1013C0000248806E002818BF00477047CC0B0020F1
:1013D0000248406E002818BF00477047CC0B002021
:1013E0000248006F002818BF00477047CC0B002050
:1013F0000248406F002818BF00477047CC0B002000
:101400000248806F002818BF00477047CC0B0020AF
:101410000348D0F89400002818BF00477047000028
:10142000CC0B00200348D0F89800002818BF0047D4
:1014300070470000CC0B00200348D0F89C00002827
:1014400018BF004770470000CC0B00207047000019
:101450000248C06C002818BF00477047CC0B002022
:101460000248006D002818BF00477047CC0B0020D1
:1014700002480068002818BF00477047CC0B0020C6
:101480002A2828BF704770B504460D46FEF774FE43
:10149000034941F82450BDE87040FEF771BE0000DA
:1014A000CC0B00200100084804BFC02100F036BA70
:1014B000012904BF402100F031BA022904BF802174
:1014C00000F02CBA704700000010014070B50446CF
:1014D000164D284600F01FFA9CB1012C16D0022CA4
:1014E00018BF70BD10F0800F4FF0800128461CBF60
:1014F000BDE8704000F012BA04BFBDE8704000F0D3
:101500000FBA0120FFF7E2FF0224E1E710F0400FDD
:101510004FF0400128461CBFBDE8704000F0FEB906
:1015200004BFBDE8704000F0FBB9000000100140AE
:10153000244901222F281CD022DC242819D013DCB6
:10154000082833D008DC072828BF7047DFE800F000
:101550002E2E2E172E172E000A2827D020281EBF29
:1015600022282328704704E0A0F12503092B88BF17
:1015700070478B69203802FA00F018438861704781
:1015800040381E2828BF7047DFE800F016161616F0
:1015900016160F0F0F0F0F160F0F16160F16161623
:1015A000161616160F160F161616E8E74B6902FAEE
:1015B00000F0184348617047CB6902FA00F0184305
:1015C000C8617047001002402DE9F041102836D262
:1015D000DFE800F05858585808131E585858585803
:1015E00058585829FEF7C8FD27490A6842F4803246
:1015F0000A60BDE8F041FEF7C3BDFEF7BDFD22491C
:101600000A6842F400320A60BDE8F041FEF7B8BD56
:10161000FEF7B2FD1C490A6842F480220A60BDE868
:10162000F041FEF7ADBDFEF7A7FD4FF0E0210A69DE
:1016300042F001020A61BDE8F041FEF7A1BD4FF0A2
:10164000E02671680127491C07EB4111C9B28842A5
:1016500028BFBDE8F081A0F11001CA1701EBD261EB
:10166000C1F34714103821F01F01451AFEF784FD1D
:1016700007FA05F106EB8402C2F80011BDE8F0415B
:10168000FEF77EBDBDE8F08124ED00E0034910F0D7
:10169000805F0CBF4860C1F804047047000002403E
:1016A000002901680CBF21F0010141F00101016036
:1016B000704700000268002122F001020260016010
:1016C00041608160C160334B334AC11A984204BF04
:1016D000506840F070601ED02CDC304BA0EB030152
:1016E000984204BF506840F4704014D015DC2C4977
:1016F000401801BF506840F00F0050607047142838
:1017000004BF506840F0F00005D0282818BF70478B
:10171000506840F4706050607047142904BF5068EE
:1017200040F47020F7D0282904BF506840F47000BE
:10173000F1D07047B1F56C7F04BFD2F8040440F4D7
:10174000706023D012DCB1F5627F01BFD2F80404CF
:1017500040F00F00C2F804047047B1F5677F18BF6E
:101760007047D2F8040440F0F0000FE0B1F5717F4B
:1017700004BFD2F8040440F4704007D0B1F5767F7E
:1017800018BF7047D2F8040440F47020C2F8040473
:101790007047000080000240000002404400024008
:1017A000F8FFFDBF0022064910F0805F0CBF0968FA
:1017B000D1F80014014218BF012210467047000002
:1017C00000000240002A02680CBF22EA0101114316
:1017D0000160704730B402680D6A8B68D1F810C0A0
:1017E0004C691D434CEA040C45EA0C048B69D1F8A2
:1017F0001CC01C4344EA0C044B6AD1F828C02343A4
:101800006FF30E1243EA0C031A430260CA68426087
:101810000A6882604968C16030BC704704490A6840
:1018200022F010020A600A68104308607047000046
:101830000020024004490A6802F038020A600A687F
:101840001043086070470000002002402DE9F001BD
:10185000CB78002213F0100F03F00F041CBF8B781D
:101860001C430B880F2513F0FF0F4FF0010622D009
:10187000D0F80070B1F800C006FA02F30CEA030CCD
:101880009C4514D14FEA820C05FA0CF827EA0807A8
:1018900004FA0CFC4CEA070791F803C0BCF1280FCE
:1018A00008BF436103D0BCF1480F08BF0361521C5D
:1018B000082ADFD307600A88FF2A9CBFBDE8F00131
:1018C000704747685FF0000202F10803B1F800C0FA
:1018D00006FA03F30CEA030C9C4515D14FEA820C7F
:1018E00005FA0CF827EA080704FA0CFC4CEA07078B
:1018F00091F803C0BCF1280F08BF436191F803C001
:10190000BCF1480F08BF0361521C082ADCD34760B2
:10191000BDE8F0017047C06880B270474161704710
:10192000016170477047000010B586B000F0C2F842
:10193000DFF83CC10023CCF834308CF802308CF84E
:1019400003308CF808308CF80730CCF80C30CCF829
:101950002030CCF81830CCF814308CF801308CF8EA
:1019600006300CF11B000221437000F8023F491EB3
:10197000FAD18CF804308CF80530CCF82C303D4886
:101980004FF48461CCF82430491E090400F8013B6F
:10199000090CF9D138488021491E090400F8013B9F
:1019A000090CF9D1334886460EF1580233A4046578
:1019B0004261491C58305832C9B20B29F6D32FA1C5
:1019C000436101652E48CCF828E04FF4C871CCF88B
:1019D000303000BF491E090400F8013B090CF9D161
:1019E000274886460EF11402037024A40461426065
:1019F000491C1430143289B21329F5D303701FA186
:101A000043600161CCF810E001F0B8FA1D480323EF
:101A10000022802101AC0FC44FF6FF73009300F544
:101A2000FE721F230021184800F022FA05AA17A110
:101A30001F2000F083FA194803230022802101AC03
:101A40000FC44FF6FE73009300F5FE721E230021B3
:101A5000134800F00DFA05AA12A11E2000F06EFA3C
:101A600000F029F806B0BDE81040FFF75BBF0000AA
:101A70006C00002084120020041200203F000000AF
:101A8000740C0020041000208131000875432F4F92
:101A9000532D49492049646C65000000040E002064
:101AA0009D31000875432F4F532D494920537461D0
:101AB000740000007047704770B5174CE07901283A
:101AC00018BF70BDFEF76AFBA178054621B1481E1C
:101AD00010F0FF00A0701AD1E078C0B90F48A179CA
:101AE0000F4A415C525C805C00EBC100C1B20D4802
:101AF000617150F82120E2622079814207D0D06BD9
:101B0000401CD063E068401CE060FEF763FB2846A1
:101B1000BDE87040FEF746BB6C000020B6400008F0
:101B2000880000200412002070B505460E48007899
:101B300000281CBF002070BDFEF730FB0B490C686D
:101B4000002C1CBF62680A60FEF72CFB4CB1012020
:101B500020700020208106A065602061204601F0F1
:101B600003FA204670BD00006E0000207C000020BB
:101B70003F0000002DE9F0470546007889461446ED
:101B800001281FBF012020700020BDE8F0872C48ED
:101B9000007800281FBF022020700020BDE8F087D9
:101BA0002848007800281FBF0D2020700020BDE8C5
:101BB000F087FEF7F3FA6E68824600272EB1504692
:101BC0006F60FEF7EFFA277031E0DFF87C80D8F81D
:101BD000000090F8341041F0020180F8341080F8D1
:101BE0003570C0F83090284601F08EF95046FEF767
:101BF000D9FA01F001FAFEF7D1FA8146D8F80000CF
:101C000090F83510002904BF466A277003D00229D6
:101C100010D10E202070D8F80010484681F834709A
:101C200081F83570CF610F624F62FEF7BBFA304624
:101C3000BDE8F087294601F053F90A20EAE70000E1
:101C40006E0000206F0000209000002070B5044658
:101C500000780D4601281CBF012070BDFEF79EFADA
:101C60000646A07A58B1002302222946204601F0F8
:101C7000CFF83046FEF796FA01F0BEF90AE0606848
:101C800020B13046FEF78EFA142070BD30466560F4
:101C9000FEF788FA002070BD70B505460E48007842
:101CA00000281CBF002070BDFEF778FA0B490C68B5
:101CB000002C1CBF62680A60FEF774FA4CB1032066
:101CC000207025810020606005A02061204601F081
:101CD0004BF9204670BD00006E0000207C00002003
:101CE0003F0000002DE9F04705460078884614467D
:101CF00003281EBF01202070BDE8F0872648007829
:101D0000002818BF022003D12448007818B10D2004
:101D10002070BDE8F087FEF741FA81462889002649
:101D200038B1401E28814846FEF73CFA2670BDE8CF
:101D3000F0871B4F396891F8340040F0010081F8BA
:101D4000340081F835602846C1F8308001F0DCF8B5
:101D50004846FEF727FA01F04FF9FEF71FFA8046D2
:101D6000386890F83510002908BF267003D0022982
:101D70000DD10E202070386880F8346080F835600E
:101D8000C66106624046BDE8F047FEF70BBA294639
:101D900001F0A6F80A20EDE76E0000206F00002099
:101DA0009000002070B50446007803281CBF012075
:101DB00070BDFEF7F3F90546A07A58B10023012261
:101DC0001946204601F024F82846FEF7EBF901F009
:101DD00013F909E020894FF6FF71884206D2401CB2
:101DE00020812846FEF7DEF9002070BD2846FEF768
:101DF000D9F9322070BD00000B49C879002818BFFE
:101E000070470A4A88790A4B105C1B5CD25C02EB73
:101E1000C000C0B24871074A087152F82000C86279
:101E20004862FEF7C2B900006C000020B64000080E
:101E3000880000200412002010B5022000F070F984
:101E4000FEF7ACF9084C00212162FEF7ABF96420E3
:101E500000F066F9FEF7A2F9216A61610121617063
:101E6000BDE81040FEF79EB96C000020FEF7C4BF2D
:101E70002DE9FF4F83B01C46DDF84CB0DDF840A0E3
:101E8000DDF84890DDF84480149DFEF787F9264977
:101E9000097829B1FEF786F93C2007B0BDE8F08F3C
:101EA000224E56F82410002937D1012146F824107B
:101EB000FEF778F94146484615F0010F4FF000074C
:101EC0001CBF15F0020F002803D0401E41F8047B10
:101ED000FBD12B46059A0499039800F099F8014626
:101EE000534642462046CDF804B0CDF80090029506
:101EF00001F0C0F8050006D10D480078012808BFA0
:101F000001F07AF805E0FEF749F946F82470FEF78B
:101F100049F9284607B0BDE8F08FFEF743F92820BD
:101F200007B0BDE8F08F00006E0000200412002012
:101F300073000020FEF761BFFEF761BF70B5054674
:101F400010480E4600781446002818BF122017D1FA
:101F5000FEF724F9FF2D02BF0B49096891F83650AE
:101F60000A4951F825104325002918BF012903D13A
:101F7000FEF718F9257070BD0E65FEF713F9002005
:101F8000207070BD6E000020900000200412002020
:101F9000FEF7AEBF2DE9F0410446002008600D4673
:101FA0004860FEF7FBF8FF2C02BF1749096891F85B
:101FB0003640164951F82410002918BF012904D1D0
:101FC000FEF7F0F84320BDE8F0810A8A12F0010F15
:101FD00004D1FEF7E7F84520BDE8F08100248F68C2
:101FE000CE68FEF7DFF83968381D21B950F8041BB8
:101FF000641C0029FAD0A0002860301B80006860B3
:102000000020BDE8F08100009000002004120020B4
:102010004FF0807342F8043910606FF00103101F15
:1020200042F8043C4FF0123240F8042D4FF00332D6
:1020300040F8042D4FF0023240F8042D521040F8C1
:10204000042D40F8041D4FF0113140F8041D11011A
:1020500040F8041D4FF0093140F8041DD10040F84C
:10206000041D4FF0073140F8041D4FF0063140F8D1
:10207000041D4FF0053140F8041D910040F8041D87
:102080007047000070B50446FEF788F81F49FF2C22
:10209000096804BF012591F8364005D091F8361043
:1020A000A14214BF00250125194951F8241019B97E
:1020B000FEF778F8482070BD012903D1FEF772F8C9
:1020C000432070BD91F83820124B91F839E013F895
:1020D00002C02CEA0E0C03F802C09A5C3AB90E4A10
:1020E00091F83A3092F800C02CEA0303137091F88B
:1020F000342042F0080281F83420FEF753F8012D15
:1021000008BF00F079FF002070BD000090000020A3
:10211000041200208800002072000020FEF7E9BEB3
:1021200010B5044613480078002818BF10BD002CD5
:1021300008BF10BDFEF732F80F49104B0A6892F83D
:10214000381092F839E013F801C02CEA0E0C03F8AD
:1021500001C0595C39B90A4992F83A3091F800C087
:102160002CEA03030B701463FEF71CF8BDE8104063
:1021700000F042BF6E000020900000208800002088
:1021800072000020DFF878C09CF800C0BCF1000F9E
:102190001CBF5520704710B54FF47A7C03FB0CF33D
:1021A000B3FBFCF34FF4616C00FB0CF0C1EB0111CD
:1021B00000EB810010447D21484313EBC0041DD087
:1021C000FDF7ECFF0F49104B0A6892F8381092F8AF
:1021D00039E013F801C02CEA0E0C03F801C0595C79
:1021E00039B90A4992F83A3091F800C02CEA030351
:1021F0000B701463FDF7D6FF00F0FEFE002010BD4B
:102200006E00002090000020880000207200002056
:1022100010B5FDF7C3FF03490C68FDF7C3FF204667
:1022200010BD0000A00000202DE9F04100F056F89C
:10223000FDF7B4FF274F796B491C7963FDF7B2FFB7
:10224000F879012818BFBDE8F081787A01250026C9
:1022500038B1012808BFBDE8F08102280CBF7D72AB
:102260007E723C6B94F836001F2808BFBDE8F081F1
:10227000DFF86480FDF792FF216B11B3491E2163E3
:102280001FD194F8341011F0370F0FBF84F8356068
:1022900021F0370184F8341084F8355094F8341064
:1022A00011F0080F0DD194F83A10BA791143B971B1
:1022B00094F8381094F8392018F801301A4308F8C7
:1022C00001206469FDF76EFF94F836001F28D1D114
:1022D000BDE8F0816C00002088000020FEF70BBEF6
:1022E0002DE9F047FA4EDFF8E483307988B0411CDD
:1022F00018F80000C9B20027317143280CD118F832
:102300000100491C3171716A002918BF8847378262
:10231000002008B0BDE8F087328A002A1EBF0020E6
:1023200008B0BDE8F08702220125EA4C542804BF1A
:102330002070358200F0438231DC322800F02682A2
:1023400011DC002800F00782312840F0388220702C
:10235000358200F0D1FA317918F80120491C317129
:10236000027000F02CBA342800F02182532840F08B
:1023700026822070358218F80100491C3171D64937
:10238000002808BF0D7000F01A82012808BF0F70E6
:1023900000F01582022808BF0A7000F010BADFF8BA
:1023A0003C93732823D00DDC622800F0A3816C28B5
:1023B00040F0058220707420607032820025C84F82
:1023C00000F072B974286DD0772840F0F881207041
:1023D000358200F091FA317918F80120491C3171E9
:1023E000511EB1F1FF3F40F3EA8100F09DB920702A
:1023F0003582FFF70DFF0746000C00F077FCB8B2FE
:1024000000F074FCD9F80070380C00F06FFCB8B222
:1024100000F06CFC4FF4907000F068FC308A80286B
:102420003EBF2554401C30821E216846FEF776F9D7
:10243000684600F0C9F99DF80020002069462AB1DD
:10244000401C11F8012FC0B2002AF9D1318A80292D
:102450003EBF6054491C31826A46002100280DD9D4
:10246000338A92F800C0802B3EBF04F803C05B1C87
:102470003382521C491CC9B28142F1D300F0CEF91B
:102480000446000C00F032FCA0B200F02FFC00F07B
:10249000C7F90446000C00F029FCA0B200F026FCAD
:1024A00000F08DB92070358200F026FA0546FDF760
:1024B00075FE824600F056FB31893081411AB069C1
:1024C00089B200EB01085046C6F81880FDF76AFE95
:1024D0004FEA184000F00AFC1FFA88F000F006FCF2
:1024E000002D18BF012D7DD0D9F80000854207D1FD
:1024F000696C286CA8EB01010844C5F84480286485
:102500002B6D00211A001CBF1078002805D0481C34
:10251000C1B212F8010F0028F9D1308A80283EBFDD
:102520002154401C3082002200290DD9308A93F8B2
:1025300000C080283EBF04F800C0401C30825B1CF5
:10254000501CC2B28A42F1D3308A95F836108028E6
:102550003EBF2154401C308295F8340018B9296BD5
:10256000002918BFF020318A80293EBF6054481CE2
:102570003082EC69200C00F0B9FBA0B200F0B6FB91
:102580002C6B200C00F0B2FBA0B200F0AFFB2C6C67
:10259000200C00F0ABFBA0B200F0A8FBEC6B200C11
:1025A00000F0A4FBA0B200F0A1FBAC6C200C00F08A
:1025B0009DFBA0B200F09AFBE8688400200C00F0BC
:1025C00095FBA0B200F092FBEC6C200C00F08EFBAF
:1025D000A0B200F08BFB2C68200C00F087FBA0B2AF
:1025E0005AE0FFE73FA200201146401C11F8013FCE
:1025F000C0B2002BF9D1318A80293EBF6054491CFA
:102600003182002100280DD9338A92F800C0802B36
:102610003EBF04F803C05B1C3382521C491CC9B284
:102620008142F1D3308A802808D22754401C80B2DE
:10263000308280283EBF2754401C3082384600F04C
:1026400055FB384600F052FB384600F04FFB384649
:1026500000F04CFB384600F049FB384600F046FBE2
:10266000384600F043FB384600F040FB384600F0A7
:102670003DFB384600F03AFB384600F037FB384661
:1026800000F034FB384600F031FB384600F02EFBFA
:10269000384600F02BFB384600F028FBFFF7B8FD6A
:1026A00080B200F023FB8AE057F82540002C18BFC9
:1026B000012C05D0200C00F019FBA0B200F016FB95
:1026C000681CC5B2202DEFD379E00000F41600207D
:1026D000A800002074170020750000209000002042
:1026E00004120020494E56414C4944205441534B5A
:1026F000210000002070358200F0FEF8317918F8D2
:102700000120491C3171511EB1F1FF3F57DD328A62
:102710000378802A3EBFA354521C3282401C491EBB
:10272000B1F1FF3FF3DC4AE00388328A4FEA132C11
:10273000802A3EBF04F802C0521C3282DBB2328AC9
:10274000802A3EBFA354521C3282801C491EB1F124
:10275000FF3FE9DC33E02070358200F0CDF805461C
:10276000307918F80010401C4C1E3071B4F1FF3F56
:1027700025DD2F68380C00F0B9FAB8B200F0B6FACF
:102780002D1D641EB4F1FF3FF3DC18E0207035828C
:1027900000F0B2F8317918F80120491CC9B218F8D4
:1027A0000130491C317143EA0221018007E02070A9
:1027B000358200F0A1F8044600F09EF82060308ACF
:1027C00008B0C0B2BDE8F08770B50546FEF795FBCE
:1027D00009491E22B0FBF1F0C4B208A12846FDF75A
:1027E000C4FF0A21B4FBF1F000F1300201FB1040FC
:1027F000AA753030E87570BD40420F005354205325
:10280000544D33322028436F727465782D4D33292F
:1028100020287878204D487A290000000020704751
:1028200000207047064A00211170064A916111701C
:10283000917191819182D1715162118100F004B83E
:1028400075000020A800002010B588B0044600F0F4
:1028500063F90020ADF814000C21ADF81610ADF8A6
:1028600018004FF40071ADF81000ADF80400ADF899
:102870000810ADF81200ADF80600ADF80A00039498
:102880005220FEF755FE2320FEF752FE4FF48060E3
:10289000ADF81C0003208DF81E001820134C8DF895
:1028A0001F0007A92046FEF7D1FFE014ADF81C0079
:1028B00004208DF81F0007A92046FEF7C7FF0C4C27
:1028C00003A9204601F05DFB01A9204601F0FDFAB5
:1028D0000121204601F00BFB06492720FEF7D0FD21
:1028E0002720FEF75FFC08B010BD0000000C01407F
:1028F00000480040052A0008DFF834C00B499CF866
:1029000004000A5C401CC0B20B5C401CC0B243EA2D
:1029100002220B5C401CC0B2095C401C8CF8040015
:1029200041EA032040EA024070470000F41600200C
:10293000A800002070B52D4C0025E169491CE1611B
:102940002146897822780144C9B2062A4BD2DFE8B1
:1029500002F0030B0F1F3035ED2818BF70BD0120AA
:102960002070E570257170BD8C283CD1022023E0D9
:10297000002808BF012104D00021802888BF01223F
:1029800000D8002211432ED1A0706070032013E004
:10299000E278802A03D2164B9854501CE070A17044
:1029A0006078401E10F0FF00607018BF70BD0420FA
:1029B00002E0A170B9B90520207070BD8D2812D138
:1029C0006089401C6081FFF78BFC60B1A081FDF73E
:1029D000E5FB0646E07918B900F0CEF800F07EF984
:1029E0003046FDF7DFFB257070BD0000A800002019
:1029F000F4160020012240F22551014801F0A9BA45
:102A00000048004010B5FDF7B7FB14490A78521C86
:102A10000A70FDF7B5FB124840F22551044601F05B
:102A200076FA50B1204601F0EFFAC0B2FFF782FF0C
:102A300040F22551204601F041FA40F2277120462C
:102A400001F065FA30B100F097F840F227712046A6
:102A500001F034FABDE81040FFF72EB86E000020F8
:102A60000048004070B50546FDF798FB064600F0AB
:102A700079F8084A014613891181C01A83B2906916
:102A8000C41830469461FDF78DFB00206C64286407
:102A900070BD0000A800002070B5FDF77FFB054663
:102AA00000F060F80B4A014613891181C01A83B205
:102AB0009069C41828469461FDF774FB06480068C5
:102AC000426C016CA21A1144016404480068446419
:102AD00070BD0000A8000020900000209800002099
:102AE0000149486270470000A800002010B5FDF7BA
:102AF00055FB044600F036F806490A890881821A17
:102B0000886992B2104488612046BDE81040FDF704
:102B100049BB0000A800002000B583B04FF6FF704D
:102B2000ADF804000020ADF80000ADF80600ADF8E7
:102B300002000121084600F08FFB69464FF08040FB
:102B400001F02EF900214FF0804001F027F9012219
:102B50001102880501F01FF90121880701F00EF923
:102B600003B000BD4FF0804001F013B901460148A9
:102B700001F04EBA004800402DE9F041504C0426C7
:102B80002046A3798189828A0025C089092B79D2C0
:102B9000DFE803F00519273179834755620051EAD0
:102BA000020002BFE571BDE8F04100F08FB88C2053
:102BB000FFF7DCFF206A401C20620120E071A07159
:102BC000E581BDE8F081ED20FFF7D0FF206A401CD1
:102BD0002062A08900280CBF06200220A071BDE859
:102BE000F081C8B2FFF7C2FF206A401C20620320B8
:102BF000A071A08920E033490F5C3846FFF7B6FF8B
:102C0000206A401C2062607938446071E089401C71
:102C100080B2E081A189884224BFA671A581BDE868
:102C2000F081501CC0B2FFF7A1FF206A401C206257
:102C30000720A071A08A401C6071BDE8F08143208C
:102C4000FFF794FF206A401C20620820A071607981
:102C500043306071BDE8F0811B490F5C3846FFF7D7
:102C600085FF206A401C2062607938446071E089E9
:102C7000401C80B2E081A18A884224BFA671A5824F
:102C8000BDE8F08116E06079FFF770FF206A401C14
:102C900020620520A071BDE8F0818D20FFF766FF5E
:102CA000206A401C2062A5712582608A401C6082D7
:102CB000BDE8F081A571E571BDE8F04100F006B80E
:102CC000A800002074170020F4170020002240F212
:102CD0002771014801F03DB900480040012240F24F
:102CE0002771014801F035B900480040DFF828C0DD
:102CF000020ABCF81010094B80293EBF5A54491CE7
:102D0000ACF81010C1B2BCF8100080283EBF1954B6
:102D1000401CACF810007047A80000207417002079
:102D20002DE9F04106460F4600F098F90546802847
:102D300022BF7F25002086F87F001C4CA08A00B3AC
:102D4000002F08BFBDE8F081E08A411CE1823846CF
:102D5000FFF7E6F9A08A0028F6D1A582314614488B
:102D6000FDF749FDA08A002808BFBDE8F081FDF706
:102D700015FA0546E079A0B9FFF7FEFEFFF7AEFFB2
:102D80000FE0A58231460A48FDF735FDA08A0028EC
:102D900008BFBDE8F081FDF701FA0546E07900289B
:102DA000EAD02846BDE8F041FDF7FCB9A8000020B4
:102DB000F417002000B585B0684600F083FA00984B
:102DC00005B000BD10B5FDF7E9F906490A78521CB7
:102DD0000A70FDF7E7F9FFF727FABDE81040FEF7A4
:102DE0006BBE00006E00002010B5FFF7E3FF4FF44C
:102DF0007A71B0FBF1F0411E4FF0E02041610169B2
:102E000041F005010161016941F00201016110BD5C
:102E10002DE9F001847ADFF8BCC000261CF80450CC
:102E20004419E47A1CF804C00CEBC50C0CF0FF0448
:102E3000DFF8A4C05CF824C0CCF83060CCF82410D3
:102E40009CF8341091438CF83410C9B28CF83530AA
:102E500011F0080F0CD121499CF83A308E7901F11C
:102E60001C0233438B71515D9CF839301943515525
:102E70009CF838109CF839300144CA7A9A43CA72D7
:102E8000D1B221B9817A9CF83A2091438172DCF861
:102E90002020DAB19CF838609CF83A709CF83950E0
:102EA000116889B18B1993F80B8028EA050883F81B
:102EB0000B8008F0FF03002B02BF8B7ABB438B72A1
:102EC00052F8041F0029EDD1CCF81C002046BDE8C3
:102ED000F0017047B6400008041200206C0000208A
:102EE00090F8382090F839C00A44D37A23EA0C03CA
:102EF000D372DAB2002A18BF70478A7A90F83A0083
:102F000022EA00008872704710B4DFF858C000F160
:102F10000B02DCF82410C86191F8383091F83910B0
:102F20009C5C21439954DCF82410827A91F83A3061
:102F30001A43827291F838000CF11C02135C91F86C
:102F40003940A3431354105C00281CBF10BC7047C9
:102F500091F83A009CF8061021EA00008CF806006F
:102F600010BC70476C000020002200F80A2F0221DC
:102F7000427000F8022F491EFAD1704710B5502157
:102F8000144800F02DF8134A002302F110011370C9
:102F900011A05160D0600846103113740FF2380C44
:102FA000C2F81CC05161103182F820300FF2280C99
:102FB000C2F82CC05162103182F83030516306A142
:102FC000D16382F8403004A14363C16303480260C7
:102FD00010BD0000A41600203F000000A400002047
:102FE000002908BF70470022491E090400F8012B80
:102FF000090CF9D17047000010B5FDF7CFF8134B5D
:1030000004469878002804BFD878002818D11048C2
:103010009979104A415C525C805C00EBC100C1B2FE
:103020000D48597150F82120DA621879814207D091
:10303000D06B401CD063D868401CD860FDF7C5F841
:103040002046BDE81040FDF7ADB800006C00002040
:10305000B6400008880000200412002002780021F9
:103060002AB1491C10F8012FC9B2002AF9D108462B
:10307000704700002DE9FF5F06460D469346DDF8D8
:1030800040A0DDF83C90DDF83880FDF787F8384F38
:10309000BC6A002C66D06169B962FDF783F82560CF
:1030A00084F83660002584F8345084F83550C4F82C
:1030B00008B0C4F80490C4F80C802563A4F810A0EC
:1030C0000398608284F83B50F00884F8380006F0DA
:1030D000070084F8370094F83820012101FA02F241
:1030E00084F83A2001FA00F084F83900E56125629D
:1030F000A5626562E56365642564A5641DA0E56459
:103100002065002004EB8001401C4D6510F0FF009D
:10311000F8D02046FEF7AAFE2046FEF70BFFFDF78B
:103120003DF8154941F82640396BA56161610029D8
:1031300018BF8C613C6394F83A10BA791143B971A5
:1031400094F838100D4A94F839C0535C43EA0C03E4
:103150005354397A491C3972FDF724F8002004B021
:10316000BDE8F09FFDF71EF8422004B0BDE8F09FD7
:103170006C0000203F0000000412002088000020A6
:1031800010B5054CFDF70AF8216A491C2162FDF7CC
:1031900009F8FEF7D1FEF5E76C000020F0B5214FED
:1031A00083B0787828B9C820FEF7BAFF787800286D
:1031B000F9D078696421B0FBF1F00026786100282D
:1031C00002BF3E70FF20FEF75DFF174DFCF7E6FFE4
:1031D000396A3E62B961FCF7E5FF7969B869B0FB0D
:1031E000F1F0C0F164003870FEF7D2FE002401A9AE
:1031F0002046FEF7CFFE60B955F82400002818BF1E
:10320000012806D0C268816801EB820181640299BD
:10321000C164601CC4B2202CE9D36420FEF780FF97
:10322000D4E700006C00002004120020034A51681B
:1032300021F44041084350607047000000100240F4
:10324000044A002951690CBF21EA0000084350617B
:103250007047000000100240044A0029D1690CBFE9
:1032600021EA00000843D0617047000000100240CE
:10327000044A002991690CBF21EA000008439061CB
:1032800070470000001002400C48016841F0010145
:10329000016041680A4A11404160016821F410212F
:1032A00021F080710160016821F480210160426891
:1032B000002122F4FE02426081607047001002404B
:1032C0000000FFF810B4264A5168264B11F00C019B
:1032D00018BF042901D0082901D0036017E0516804
:1032E0004FF0020C01F470110CEB9141D2F804C0C4
:1032F0001D4C1CF4803F04BF6143016007D0D2F82D
:1033000004C01CF4003F0CBF594361430160516885
:10331000DFF858C001F0F00109091CF8011003683A
:1033200023FA01F14160536803F4E0631B0A1CF8BF
:10333000033021FA03F38360536803F46053DB0A1C
:103340001CF80330D940C1605268ACF1040302F4A8
:103350004042920B9A5CB1FBF2F1016110BC7047E4
:103360000010024000127A0000093D00A64000084B
:1033700000224109094B012908BF196803D002291D
:1033800014BF596A196A00F01F00012303FA00F004
:10339000084218BF0122104670470000001002408A
:1033A0000248406800F00C00704700000010024026
:1033B000034A516821F0F001084350607047000053
:1033C000001002400C490A6822F480320A600A6840
:1033D000B0F5803F22F480220A6004BF086840F400
:1033E000803006D0B0F5802F18BF7047086840F4D1
:1033F000A02008607047000000100240034A516896
:1034000021F4E06108435060704700000010024062
:10341000034A516821F4605141EAC000506070478E
:103420000010024001490866704700000000424257
:10343000034B5A68084322F47C12104358607047CB
:1034400000100240034A516821F003010843506014
:1034500070470000001002400E4B0F4940F2FF1C65
:103460001A68002012F4003F18BF01200870486855
:10347000401C4860087810B948686045F0D1196868
:10348000002011F4003F18BF0120002818BF0120C0
:103490007047000000100240640000202DE9F00198
:1034A0002D4A2E4BDFF8ACC05361C2F810C09361B7
:1034B0004478057BC4F3C301002904F00706C5F373
:1034C000820502BF0320BDE8F0017047244C0A27A3
:1034D000615C244CDFF89080614391FBF7F158F870
:1034E00026608078B1FBF6F11926704301EB80006D
:1034F000A8F108011061495D4143516115788DB90A
:10350000642569436843C908C0085161106160457A
:1035100088BF604610611846994288BF0146084638
:10352000516106E07843C008106101FB07F0C00854
:10353000506113694FF4FA514B434843B0FBF4F028
:10354000B3FBF4F3506113619061BDE8F00100201A
:1035500070470000E86E03007418002044950800CE
:10356000E043000880A81201C04300080120704712
:1035700000B583B0012819BF00208DF80900012093
:103580008DF8080001AB012202A93B2000F0D5FA1A
:1035900000281CBF03B000BD9DF80400002818BF20
:1035A000122003B000BD000002460020002908BF21
:1035B0007047064B12F801CB491E8CEA102C33F8E9
:1035C0001CC08CEA002080B2F4D17047B6410008DC
:1035D00030B482B08DF80000081D002210F801CC34
:1035E0006946022310F8024D81F801C010F801CCA1
:1035F00001F8024F5B1EF5D100246D46002015F83E
:1036000004C004215206120E0CFA00F3534013F0CA
:10361000800318BF09235A405206120E431C0CFAAD
:1036200003F3534013F0800318BF09235A40801C52
:10363000491E11F0FF01E5D1601CC4B2052CDDD399
:10364000012002B000EB420030BCC0B27047000065
:1036500010B586B001211420FFF70AFE01210803EE
:10366000FFF706FEE020ADF8140003248DF81640A5
:1036700018208DF8170005A91E48FEF7E7F810205E
:10368000ADF814008DF816401B4C8DF8170005A9F5
:103690002046FEF7DBF810212046FEF741F9002016
:1036A000ADF804004FF48271ADF80610ADF80800D3
:1036B0000221ADF80A100121ADF80C104902ADF855
:1036C0000E103021ADF81010ADF8120007200B4C91
:1036D000ADF8140001A9204600F0FFFA0022712184
:1036E000204600F0E9FA0121204600F0D5FA06B0A4
:1036F00010BD0000000801400010014000300140F2
:103700002DE9F041694E86B0306848B90120FEF7D6
:10371000C3FA3060002802BFA02006B0BDE8F081E7
:1037200004AA0021FEF7DEFAFFF792FFFFF71EFF63
:10373000012818BF012440F0B28000F073FAC820BD
:1037400000F0EDF900F074FA042000F0E8F95848B0
:10375000401EB0F1FF3FFBDC00F0D6F9040040F062
:103760009E800025534F2C464FF0010804950122FE
:1037700002AB04A9104600F0E0F9002828D19DF81A
:103780000800641C10F0010F03D0B4F57A7FEED965
:1037900002E0B4F57A7F01D3342019E002AB0122B4
:1037A00004A9372000F0C9F990B902AB012204A99D
:1037B000292000F0C2F9002818BF062008D19DF882
:1037C000080010F0FE0F14BF87F800803D702846F7
:1037D000040064D105A9042000F04EF904005ED174
:1037E0009DF81500302131EA000018BF042456D19D
:1037F0000120FFF7BDFE040051D14FF4007000F02E
:10380000F3F904004BD101A9102000F0E1F80028E1
:1038100018BF044639D101A8FFF740FE9DF8090002
:1038200000F00F0008FA00F0B8609DF80A009DF85B
:103830000B108007000D00EB81009DF80C1000EBD1
:103840009110411C9DF80D008007420F9DF80E005D
:1038500002EBD012921C91407960397801290BD18A
:10386000C0F3840180079DF80F20C00E491C00EBB7
:103870005210401C484306E080069DF80F10400E91
:1038800000EBD110401C2C46F86044B93068FEF7BC
:1038900089FA00F0D3F9002006B0BDE8F081306865
:1038A000FEF780FA204606B0BDE8F081D000002087
:1038B0003F420F0074180020F8B5154C05460E461F
:1038C00017466A4600212068FEF70CFAFFF74EFE05
:1038D000012804D02068FEF765FA0120F8BD0D48E4
:1038E0004068A84204D22068FEF75CFA0520F8BDC3
:1038F000284600F0E8F8050004D13946304600F0CB
:103900000BF805462068FEF74DFA2846F8BD000082
:10391000D0000020741800202DE9F04106460F4623
:1039200000244FF4807500F07DF900BF00F0FAF933
:10393000641CFF2801D1AC42F8D3B4F5807F0CD3CE
:103940002248002405690120FEF7EAFB00F0EAF9AD
:10395000641CFF2801D1AC42F5D3AC4204D300F083
:1039600067F93120BDE8F081FE2807D0FF2000F084
:10397000F3F900F05DF92120BDE8F0810024002E6C
:1039800006D900BF00F0CEF93855641CB442F9D313
:1039900000F0C8F9044600F0C5F900EB0424B1B208
:1039A0003846FFF701FEA0424FF0FF0006D000F0BE
:1039B000D3F900F03DF92020BDE8F08100F0CCF90A
:1039C00000F036F90020BDE8F081000074180020F6
:1039D000F0B583B006460D46002701AB012202A9CF
:1039E0000920029700F0A9F800281CBF03B0F0BD21
:1039F0009DF8040000281EBF122003B0F0BD002473
:103A000000F010F900F08EF9641CFF2802D1082C98
:103A1000F8D301E0082C04D300F00AF9312003B0F8
:103A2000F0BDFE280EBF002428700124B44205D248
:103A300000F078F92855641CB442F9D300F072F90B
:103A4000044600F06FF900EB042431462846FFF7E6
:103A5000ABFDA0424FF0FF0006D000F07DF900F072
:103A6000E7F8202003B0F0BD00F076F900F0E0F8B0
:103A7000384603B0F0BD000010B584B000200C46FD
:103A8000039001AB042203A93A2000F056F8002865
:103A90001CBF04B010BD9DF8040000281EBF1220FA
:103AA00004B010BD01A8611E9DF805305FF0020250
:103AB00010F802CF4B70437801F802CF521EF7D1B5
:103AC000002004B010BD10B582B04002010E8DF888
:103AD0000710010C8DF80610000A8DF8050000246F
:103AE0008DF804406B46012201A9112000F025F851
:103AF00000281CBF02B010BD9DF8000000280CBFBC
:103B00002046122002B010BD00B583B0002001ABEA
:103B1000012202A9029000F010F803B000BD70B5B8
:103B2000051E4FF0000498BF70BDFF2000F014F98F
:103B3000601CC4B2AC42F8D370BD2DE9F04104461C
:103B40000E4690461D4600F06DF804F03F0747F022
:103B5000400000F001F90324305D00F0FDF8641E20
:103B6000B4F1FF3FF8DC47F040003146FFF730FD8D
:103B700000F0F2F8B8F1010F14BFB8F1020F0126FE
:103B800008D0B8F1030F08BF022603D0B8F1040F24
:103B900002D10526002407E0FF2000F0DDF800F048
:103BA00047F81020BDE8F08100F0BCF8641C10F06C
:103BB000800F02D0642CF7DB01E0642C04DB00F002
:103BC00037F81120BDE8F081741EB4F1FF3F06DD27
:103BD000285500F0A7F8641EB4F1FF3FF8DC00F0B0
:103BE00027F80020BDE8F08100B583B0010E8DF804
:103BF0000B10010C8DF80A10010A8DF809108DF8D0
:103C0000080001AB012202A91020FFF796FF00284F
:103C10001CBF03B000BD9DF80400002818BF12208F
:103C200003B000BD10210148FDF778BE001001402F
:103C300010210148FDF774BE0010014010B586B098
:103C40000020ADF804004FF48271ADF80610ADF815
:103C500008000221ADF80A100121ADF80C1049024C
:103C6000ADF80E100821ADF81010ADF812000720C5
:103C7000084CADF8140001A9204600F02EF80022EF
:103C80007121204600F018F80121204600F004F8C8
:103C900006B010BD00300140002901880CBF21F0A2
:103CA000400141F040010180704702461289002026
:103CB0000A4218BF012070470909012303FA01F1E4
:103CC000002A828889B20CBF22EA01011143818057
:103CD0007047808970478181704730B402880B88B3
:103CE0004D88B1F804C0CC881D434CEA040C0B8904
:103CF00045EA0C04B1F80AC01C438B8944EA0C0461
:103D0000B1F80EC0234302F4415243EA0C031A43B4
:103D10000280828B22F400628283098A018230BC95
:103D20007047000010B50B4C02212046FFF7BDFF85
:103D30000028F9D0FF212046FFF7CDFF01212046C2
:103D4000FFF7B3FF0028F9D02046FFF7C2FFC0B24B
:103D500010BD00000030014070B5074C054602213F
:103D60002046FFF7A2FF0028F9D029462046BDE8EB
:103D70007040FFF7B0BF000000300140002901880B
:103D800006BF21F0010121F47C4141F001010180D5
:103D90007047808C704701858282704781847047AC
:103DA000028802F08F020280CA884B88B0F800C0F7
:103DB0001A4342EA0C0202808A88012382850A881B
:103DC000A0F1804CBCF5963C0285838219BFA0F11E
:103DD0008042B2F59A32097A0186704770B5184C64
:103DE000184D194E9AB06A460021A068FDF7C2FE30
:103DF000007831280BD0322813D1327813A101A8D2
:103E0000FCF776FC012101A8FEF78AFFEBE72A7890
:103E100013A101A8FCF76CFC012101A8FEF780FFAB
:103E2000E1E7012113A0FEF77BFF012115A0FEF7BA
:103E300077FF012118A0FEF773FF012119A0E3E726
:103E4000000000206C000020740000200A23546150
:103E5000736B73202020203D202533750A0000005D
:103E60000A435055205573616765203D2025337501
:103E700025250A000A0A4D69637269756D2C20496F
:103E80006E632E000A313A20435055205573616706
:103E900065202825290000000A323A202354617346
:103EA0006B7300000A3F3A2048656C702028546804
:103EB0006973206D656E75290A000000090A0122E8
:103EC00002FA01F1C9430180704710B4028A4FF22F
:103ED000FF031A400B88B1F802C08C88C98843EAF6
:103EE0000C03214319431143018210BC7047002980
:103EF00081890CBF21F4005141F400518181704748
:103F00000246128800200A4218BF0120704710B4F0
:103F100001F01F020124C1F3421304FA02F24FF030
:103F2000000C012B04BF83891A4004D0022B14BF5C
:103F3000838A038A1A40090A008804FA01F1002AD8
:103F400000EA01001CBF00284FF0010C604610BCC5
:103F50007047C1F3421301F01F014FF0010C0CFA3E
:103F600001F1012B08BF0C3003D0022B14BF143019
:103F70001030002A02680CBF22EA010111430160DF
:103F8000704730B50446008A85B00D464CF6FF7187
:103F90000840E98808432082A0894EF6F3110840C2
:103FA000A9882A8911436A8910430843A081A08AFD
:103FB0004FF6FF410840A9890843A0826846FFF7F1
:103FC00081F9A4F18040B0F59C3014BF02980398A9
:103FD00019214843296864228900B0FBF1F0B0FB45
:103FE000F2F109010B096FF0180C03FB0CFC3223F2
:103FF00000EB8C0003EB0010B0FBF2F000F00F00C0
:104000000843208105B030BD8088C0F308007047A8
:10401000C1F308018180704770B5074D04468021C7
:104020002846FFF76DFF0028F9D0E1B22846FFF7D8
:10403000EFFF204670BD00000038014000B587B09A
:10404000FDF7AEF8FDF770FC03230022CDE9032352
:104050000B484FF4007100F2FC7202910190009342
:1040600000210848FDF704FF069006AA06A10320D8
:10407000FDF764FFFDF7C0FE002007B000BD0000A3
:10408000EC000020010E000853746172742054612A
:10409000736B000010B5FCF76FFD4FF0000101607D
:1040A00010BD020406080000000001020304010222
:1040B00003040607080900000100020001000300D4
:1040C00001000200010004000100020001000300E1
:1040D00001000200010005000100020001000300D0
:1040E00001000200010004000100020001000300C1
:1040F00001000200010006000100020001000300AF
:1041000001000200010004000100020001000300A0
:10411000010002000100050001000200010003008F
:104120000100020001000400010002000100030080
:10413000010002000100070001000200010003006D
:104140000100020001000400010002000100030060
:10415000010002000100050001000200010003004F
:104160000100020001000400010002000100030040
:10417000010002000100060001000200010003002E
:104180000100020001000400010002000100030020
:10419000010002000100050001000200010003000F
:1041A0000100020001000400010002000100030000
:1041B0000100020001000000211042206330844011
:1041C000A550C660E770088129914AA16BB18CC1E6
:1041D000ADD1CEE1EFF13112100273325222B5525D
:1041E0009442F772D662399318837BB35AA3BDD336
:1041F0009CC3FFF3DEE36224433420040114E6642D
:10420000C774A44485546AA54BB528850995EEE585
:10421000CFF5ACC58DD55336722611163006D7763C
:10422000F6669556B4465BB77AA719973887DFF7D5
:10423000FEE79DD7BCC7C448E5588668A778400804
:10424000611802282338CCC9EDD98EE9AFF9488925
:1042500069990AA92BB9F55AD44AB77A966A711A9C
:10426000500A333A122AFDDBDCCBBFFB9EEB799B75
:10427000588B3BBB1AABA66C877CE44CC55C222CEC
:10428000033C600C411CAEED8FFDECCDCDDD2AADC5
:104290000BBD688D499D977EB66ED55EF44E133E7C
:1042A000322E511E700E9FFFBEEFDDDFFCCF1BBF15
:1042B0003AAF599F788F8891A981CAB1EBA10CD1EF
:1042C0002DC14EF16FE18010A100C230E3200450F7
:1042D000254046706760B9839893FBA3DAB33DC36A
:1042E0001CD37FE35EF3B1029012F322D232354247
:1042F000145277625672EAB5CBA5A89589856EF5FA
:104300004FE52CD50DC5E234C324A0148104667496
:10431000476424540544DBA7FAB79987B8975FE749
:104320007EF71DC73CD7D326F2369106B0165766E6
:104330007676154634564CD96DC90EF92FE9C899D1
:10434000E9898AB9ABA94458654806782768C01836
:10435000E1088238A3287DCB5CDB3FEB1EFBF98BA9
:10436000D89BBBAB9ABB754A545A376A167AF10A86
:10437000D01AB32A923A2EFD0FED6CDD4DCDAABDB9
:104380008BADE89DC98D267C076C645C454CA23CD6
:10439000832CE01CC10C1FEF3EFF5DCF7CDF9BAF89
:1043A000BABFD98FF89F176E367E554E745E932E26
:1043B000B23ED10EF01E0000010204081020408021
:1043C00000CA9A3B00E1F5058096980040420F0034
:1043D000A086010010270000E80300006400000030
:1043E000000A0C0D0F14191E23282D32373C46509D
:1043F00004000008000000000000000200010000AE
:1044000010303132333435363738396162636465A0
:10441000660030313233343536373839414243441F
:10442000454600004444000800000020D40000007D
:104430003401000818450008D4000020B01800001E
:1044400050010008000000000AD7233C00000000D3
:10445000000000000000000000000000000000005C
:10446000000000000000000000000000000000004C
:104470000000803F00000000000000000000803FBE
:104480000000803F00000000000000000000803FAE
:104490000000803F00000000000000000000803F9E
:1044A000000000000000000000000000000000000C
:1044B00000000000000000000000000000000000FC
:1044C00000000000000000000000000000000000EC
:1044D00000000000000000000000000000000000DC
:1044E00000000000000000000000000000000000CC
:1044F00000000000000000000000000000000000BC
:1045000000000000000000000000000000000000AB
:084510000000000000000000A3
:00000001FF
